:1000000000308A00AC2800000030A1001F08C3396E
:1000100021049F000D30A000A00B0C289F149F18F6
:100020000F2883161E088312A5001E08A6000430A0
:10003000A1001F08C33921049F000D30A000A00BB0
:100040001F289F149F18222883161E088312A700BA
:100050001E08A8000C30A1001F08C33921049F000E
:100060000D30A000A00B32289F149F18352883164E
:100070001E088312A9001E08AA0000343430840030
:100080000008031950280230A100A001A00B462847
:10009000A10B45289730A000A00B4C28800B4328CB
:1000A0000034B501B401B508031D6B283408253CA4
:1000B000031C6B2805150830A000A00B5D2800006C
:1000C00005110330A000A00B632800000000B40A53
:1000D0000319B50A532800340830B502031C7B28E5
:1000E000353084000310800C000803197B28792820
:1000F0000000800B7828003451200130B4003E20ED
:100100000230B400F830B5006C20B40B8228003403
:1001100051200230B400F830B5006C20B40B8B28AD
:100120000034B501B401B508031DAB283408123CF6
:10013000031CAB2805150830A000A00B9D2800006B
:1001400005110330A000A00BA32800000000B40A92
:100150000319B50A9328D02984011F3083051F1382
:1001600083161F149F141F159F15073083129F00BD
:10017000703083168F001B30650083121F138316A7
:100180001F149F141F119F151F129F161F138312F8
:100190009F171F1485120130B000B10104202608FA
:1001A000023C0318DE28FF3A031DDA282508203C0C
:1001B0000318DE28B2010330B300E2280130B20098
:1001C0000230B300A608031DE9282508323C0318B5
:1001D000EB280420E228AF0133082F020318FA2885
:1001E0008516FA30B4003E208512FA30B4003E2065
:1001F000AF0AEC28042005118512AE01300B072947
:100200000130B1073108033C031D0729B00126085E
:10021000023C03181529FF3A031D12292508203C2A
:10022000031815290530AD0046292608013C03189E
:100230002329FF3A031D20292508583C03182329A8
:100240000430AD0046292608003C03183129FF3A46
:10025000031D2E292508903C031831290330AD00D9
:100260004629A608031D38292508FA3C03183B290E
:100270000230AD004629A608031D42292508643C2A
:10028000031845290130AD004629AD01B208031D10
:100290004D29300B4D290630AD00AB01AC012808CB
:1002A000013C03185D29FF3A031D5A292708643CC5
:1002B00003185D290130AB006C292808013C031CA0
:1002C0006A29031D672927089B3C031C6A29013002
:1002D000AC006C29AB01AC01320B7329300B7329D4
:1002E0000130AB00AC005120512051200130B4004E
:1002F0003E20320B7F297C200130AE078A29B208CC
:10030000031D8A2951200230B400F830B5006C205A
:10031000B40B85292B0B90297C200130AE07912945
:1003200088202C0B97297C200130AE079829882043
:100330002D0B9B29A3292D08033C0319A3292D0864
:10034000053C031DA7297C200130AE07A829882081
:100350002D08023C0319B4292D08033C0319B429C4
:100360002D08063C031DB8297C200130AE07B929B1
:1003700088202D08043C0319C5292D08053C0319C4
:10038000C5292D08063C031DC9297C200130AE0774
:10039000CA2988200130AE05AE08031DD129912855
:1003A000D229512005112A08023C031CDE29031D15
:1003B000DD292908ED3C031CDE2985165030B400E8
:0603C0003E20FA28630054
:02400E00C43FAD
:00000001FF
